:020000040000FA
:100000005E288207003400340034013400340034A8
:1000100000340A34003400340034643400340034D2
:100020000334E8340034003427341034003401340D
:100030008634A03400340F344234403400349834D1
:100040009634803482070B340A340934073406347A
:100050000534033402348207503449344334453480
:100060004C34673465346E3400342034563465348F
:10007000723432342E3431346634003442346134D4
:100080006E34643420340034553470346434613454
:1000900074346534003449346E3469347434423411
:1000A00061346E346434003420344B3448347A3450
:1000B0000034433441344C34203400348B01073055
:1000C0009F009801831698018C019F018113FF30D6
:1000D000850086018312A901AA01AB01AC01AD0123
:1000E000752275228F22AF2237308400F0019F23C2
:1000F000C601CA010508C50003304505C400451EF8
:10010000FB21D1015330DC000030CD000301E2219E
:100110000430F000B723D200BD20D721462312308F
:10012000B5222B23C023FA2274222E214A1E9A289C
:10013000A3209528C6189E281221A028C920E820AF
:10014000FA2274229528FF305C078400C618AE2876
:100150008003801FB4280D308000B428800A0E3040
:100160000002031CB428800146231230B5222B2341
:10017000C023BD20FA22742208005C08FF3E8400E0
:1001800005300007000700070007F000840A9F23DE
:100190000800CC015C0884002E0880070330C800EA
:1001A000E220840384032F0880070230C800E22085
:1001B000840330088007840A031CDF28800A310882
:1001C000800708004C0D840A8007C80BE22808004D
:1001D00003305C07840003300002031C1129031D57
:1001E0000429840393300002031C1129031D0429F0
:1001F000840387300002031C1129031D0429840392
:1002000000300002031C11295C08840000308000CB
:10021000840A87308000840A93308000840A033087
:10022000800008002221C92003305C078400801F61
:1002300020298001840380018403800184038001DC
:1002400022210800AE09AF09B009B109AE0F2D296E
:10025000AF0F2D29B00F2D29B10A08006021050824
:10026000C500D52305084506031D2E290330450585
:10027000C300440603192E290310C40D4308C40605
:1002800044080239C7004606C601C4184F2943086E
:10029000C400D00350182E29D0182E295829023016
:1002A000C6004308C400D00A50182E29D0182E29A1
:1002B0004308C400C5195E294A165F294A1208007E
:1002C000CA18C029051DC129051A7D29851DA22925
:1002D0002030CB004A10CC23051A7B29851DA2298A
:1002E000051DC129CB03031D6B290130E221043018
:1002F000CB004A146B2901309E294A1E8329851D93
:10030000C029CA01C0298519C029CA198B292030E2
:10031000CB004A10CA15CC2385199D29051EA22998
:10032000CB0303199629CA19C0298B29CA11FF309A
:10033000E2210430CB004A148B29FF304A18BF2930
:10034000E221BF294030CB00CC23051AC0298519F2
:10035000C029CB03031DA4294A1EB82983234623A1
:100360001830B522C02346231F30B522BE23BE2934
:100370008A2346231830B5222B23BE23FA22CA0132
:100380000800CC23051ECA16051DC129CA1ECA298C
:10039000D721D329511CD02951105330DC00D32947
:1003A00051145830DC00CA01FA227422C0295308C3
:1003B000D8005408D9005508DA005608DB00520866
:1003C000D70008004D070739CD002220CE00EA21D2
:1003D000FA2208000430C800313084004D08CC00F7
:1003E0000310CC0DCC0D4C08012080008403CC0AF6
:1003F000C80BF3290800CA148030D3009630D4000B
:100400009830D5000030D600FA228C3061232D3090
:10041000B52274222E21B101B001AF010530AE002A
:100420004519142A8030AE000000C618182A22216F
:100430002E08B707031C212AB80F212AB90F212A39
:10044000BA0A2F08B807031C282AB90F282ABA0AA3
:100450003008B907031C2D2ABA0A3108BA07051E4D
:10046000092AF001373084009623CA100800A90138
:10047000AA01AB01AC01AD012030B4003708BB00CC
:100480003808BC003908BD003A08BE005C0884008A
:1004900003103B1C652A0008AA07031C542AAB0F53
:1004A000542AAC0F542AAD0A840A0008AB07031C77
:1004B0005C2AAC0F5C2AAD0A840A0008AC07031C56
:1004C000622AAD0A840A0008AD07AD0CAC0CAB0C77
:1004D000AA0CA90CBE0CBD0CBC0CBB0C5C08B40B6C
:1004E000472A0130AD000800372229308400000877
:1004F000B6000830B500B60C031C822A8615061516
:100500000611852A861106150611B50B7B2A840A69
:100510002E300402031C772A861786130800C9238D
:10052000033086000616C92306120330860006161D
:10053000CC230612033086000616CC2306120230A6
:1005400086000616CF23061220306123083061236F
:1005500001306123063061230E3061230800003032
:10056000B5220930B522BE230800CF002B20FF3969
:100570000319BE2A6523CF0A4F08B62A0800203087
:10058000B200A401A501A601A701A8015C0884008E
:100590000008A000840A0008A100840A0008A20044
:1005A000840A0008A3000310A00DA10DA20DA30D45
:1005B00003182014A40DA50DA60DA70DA80DB203B8
:1005C000031DE32A080024308400EF22840AEF226E
:1005D000840AEF22840AEF22840AEF22D32A03300E
:1005E0000007B300B319800030300007B300B31B1D
:1005F00080000800BF220230612341305118423090
:10060000652320306523270E0F39303E65232708E8
:100610000F39303E65232C306523260E0F39303ECE
:10062000652326080F39303E6523250E0F39303EED
:1006300065232E30652325080F39303E6523240EAF
:100640000F39303E652324080F39303E65232830AA
:10065000B52242230800A401A501520851185708E9
:10066000CC00CC0A0A304C02031C392BA400A50A8A
:100670003B2B4C08A4002508303E65232408303E5F
:100680006523080080304E04612308000130612397
:10069000080086018316083086008312061386162A
:1006A000FF30C10006160608C00006120000000058
:1006B000061600000612C1030319602BC019522B45
:1006C0000800BF00C9010613682BBF0049140617B4
:1006D0004923860183160030860083128612061392
:1006E00049180617F03086053F0E0F3986040616A6
:1006F00000000612F03086053F080F398604061602
:100700000000061208000430F00052085118570883
:10071000A8230800FF305C0784000008CC000530E7
:100720004C074C074C074C07F000840A0430C80003
:100730000008A823840AF00AC80B982B080004308C
:10074000C800B7238000F00A840AC80BA12B080058
:1007500083169A0070089B001C1555309D00AA3026
:100760009D009C149C18B22B1C1183120800831648
:1007700070089B001C141A0883120800C323C323AB
:10078000C323C3230800C623C6230800FF30C100CB
:10079000D72B8030C100D72B4030C100D72B203061
:1007A000C100D72B1030C100D72B0230C100FF3061
:0C07B000C200C20BD92BC10BD72B0800D4
:084000005700330043004400A7
:02400E00303F41
:10420000DF006500DC001700020050009E001B006C
:104210000000400052003600000000006C006B00FF
:104220000000A0005B009A000000E0008900D600BA
:10423000000080001F0014000100A0005900410090
:104240000100100009007C00010060002900AC00A2
:104250000100E0004400A3000000C8002200560056
:1042600000003800FF004A000000B800CD00330015
:1042700000005800F10006000000000000000000EF
:00000001FF
